:10000000A92864000C1E012899000314A4280830B4
:10001000A600A7003B088400390837193F20371D88
:1000200041203A08840038084420A001A101260894
:100030000319A428B7182C203A08840000083805B2
:10004000FF3EA00DA10DB71C2C20A60B1A282708D7
:10005000371872282008A4283B0884003908800635
:100060002008A2002108A3000030A100193063205D
:100070002208A0002308A100390880060800800497
:100080004728FF3A8005482884178004A428FF3AAF
:1000900084178005A428A000A00DA00D200D3839DC
:1000A000C1389F000030A100323063201F151F1996
:1000B0005728A1011E08A4288001840AFF3E031DC1
:1000C0005C28A428A101FC3EA000A109031C6E2805
:1000D000FF300000A00703186928A0076400A10FE3
:1000E00068280800A201A3017928A10CA00CA20D88
:1000F000A30DFF3E031875282308A1002208A000C5
:10010000A4280310A00DA10DFF3E0318812820088C
:10011000A4280310A10CA00CFF3E03188928200876
:10012000A428A20006309428A80023082102031D59
:100130009B282208200204300318013003190230E2
:100140002805031DFF30A4288313031383126400C2
:1001500008008316043099002430980083129030F0
:100160009800831602309F00FF308500E030860043
:100170008130870020308400603083128A015C2047
:10018000A030840060308A015C20E0300605E90080
:100190006908A000A10105308A018C20ED006400EF
:1001A0006D08003C8A11031DDB288A112F218A115A
:1001B000E8228A112D2964006D08013C8A11031D73
:1001C000E7288A1169218A11E8228A112D29640001
:1001D0006D08023C8A11031DF3288A11A3218A119C
:1001E000E8228A112D2964006D08033C8A11031D41
:1001F000FF288A11DD218A11E8228A112D29640045
:100200006D08043C8A11031D0B298A1143228A11AF
:10021000E8228A112D2964006D08053C8A11031D0E
:1002200017298A1197228A11E8228A112D29640040
:100230006D08063C8A11031D23298A119A228A110E
:10024000E8228A112D2964006D08073C8A11031DDC
:100250002D298A119D228A11E8228A01C5280610BB
:1002600086100611EC018A11A022061486100611D0
:100270000130EC008A11A02206108614061102300B
:10028000EC008A11A0220614861406110330EC003B
:100290008A11A0220610861006150430EC008A117F
:1002A000A0220614861006150530EC008A11A02243
:1002B0000610861406150630EC008A11A0220614DA
:1002C000861406150730EC008A11A0228A110A2331
:1002D00008008A11EE238A110A235C08EE00E60A60
:1002E0000319E70A71082C3CE4000130031CFF3EAF
:1002F000E50064007308003C8A11031D83296E0821
:10030000EB000130F3006608A0006708A100650853
:10031000A30064088A0191208A11031D98296B1893
:100320006B166B1C6B120310EB0CE601E701F20A73
:100330006400043072028A11031CA029F201F30147
:100340008A112F2308008A11EE238A110A235C08E0
:10035000EE00E60A0319E70A71082C3CE4000130BC
:10036000031CFF3EE50064007308003C8A11031D76
:10037000BD296E08EB000130F3006608A000670895
:10038000A1006508A30064088A0191208A11031D59
:10039000D2290310EB0D6B1A6B146B1E6B10E60168
:1003A000E701F20A6400043072028A11031CDA29A0
:1003B000F201F3018A112F2308008A11EE238A111A
:1003C0000A237208133C8A11031C152A8A11EB2197
:0E03D000EE008A11152A02308A007208002AF7
:1004000082070034083404340234013409340534DA
:1004100003340B3407340F340E340D340C340A34E7
:1004200009340834043402340134E60A0319E70AB3
:1004300071082C3CE4000130031CFF3EE500640021
:100440007308003C8A11031D292A6E08EB00013055
:10045000F3006608A0006708A1006508A30064080F
:100460008A0191208A11031D392AF301E601E7016F
:10047000F20A6400143072028A11031C402AF2014D
:100480008A112F2308008A11EE238A110A23720889
:10049000133C8A11031C692A8A115122EE008A1129
:1004A000692A02308A007208820701340234043457
:1004B000083409340A340C340D340E340F34073444
:1004C0000B34033405340934013402340434083461
:1004D0000034E60A0319E70A71082C3CE4000130F5
:1004E000031CFF3EE50064007308003C8A11031DF5
:1004F0007D2A6E08EB000130F3006608A000670853
:10050000A1006508A30064088A0191208A11031DD7
:100510008D2AF301E601E701F20A64001430720249
:100520008A11031C942AF2018A112F2308008A01E0
:100530002F2108008A012F2108008A012F2108009D
:1005400000308A014B20B2002108B3006C083C3E09
:1005500084003208800032308A01622001308A0132
:100560004B20B2002108B30008306C07B400B5017D
:10057000B50D34083C3E84003208800032308A01D8
:10058000622002308A014B20B2002108B3001030F3
:100590006C07B400B501B50D34083C3E8400320848
:1005A000800032308A01622003308A014B20B20081
:1005B0002108B30018306C07B400B501B50D34083C
:1005C0003C3E84003208800032308A0162200800FC
:1005D00006162430E8008A110623E8018A11062352
:1005E0000A308A016220EC01640028306C028A1112
:1005F0000318052B6C083C3E84000008E8008A11B3
:100600000623EC0A8A11031DF42A080068088A01EF
:100610000120080064308A01622007150A308A012F
:10062000622087140A308A01622087100A308A010A
:100630006220071132308A0162200730BA0001308F
:10064000B8000730BB000230B900B7018A010720AB
:10065000F00032308A0162207008DC0008006B185C
:100660006F146B1C6F10EB18EF14EB1CEF106B1971
:100670006F156B1D6F11EB19EF15EB1DEF1164007A
:100680008A116F1C542BEA0164001D306A028A1122
:100690000318542B6A083C3E8400FF30800004306D
:1006A000EA078A11031C442B64008A116F18692B16
:1006B000EA0164001D306A028A110318692B6A0876
:1006C0003C3E8400003080000430EA078A11031C9D
:1006D000592B64008A11EF1C7F2B0130EA00640063
:1006E0001E306A028A1103187F2B6A083C3E840080
:1006F000FF3080000430EA078A11031C6F2B64006E
:100700008A11EF18952B0130EA0064001E306A024E
:100710008A110318952B6A083C3E84000030800043
:100720000430EA078A11031C852B64008A116F1DAF
:10073000AB2B0230EA0064001F306A028A110318F2
:10074000AB2B6A083C3E8400FF3080000430EA078F
:100750008A11031C9B2B64008A116F19C12B023074
:10076000EA0064001F306A028A110318C12B6A086C
:100770003C3E8400003080000430EA078A11031CEC
:10078000B12B64008A11EF1DD72B0330EA006400FF
:1007900020306A028A110318D72B6A083C3E840075
:1007A000FF3080000430EA078A11031CC72B640065
:1007B0008A11EF19ED2B0330EA00640020306A0241
:1007C0008A110318ED2B6A083C3E8400003080003B
:1007D0000430EA078A11031CDD2B0800061086107E
:0E07E0000611EC018A01A0223C08F10008007D
:02400E00060F9B
:00000001FF
